:03000000021000EB
:10100000787FE4F6D8FD75816702104702170BE47C
:1010100093A3F8E493A34003F68001F208DFF48081
:1010200029E493A3F85407240CC8C333C4540F44D1
:1010300020C8834004F456800146F6DFE4800B01AB
:10104000020408102040809010F1E47E019360BCFF
:10105000A3FF543F30E509541FFEE493A360010E43
:10106000CF54C025E060A840B8E493A3FAE493A36A
:10107000F8E493A3C8C582C8CAC583CAF0A3C8C58B
:1010800082C8CAC583CADFE9DEE780BED083D082CA
:10109000F8E4937012740193700DA3A393F8740194
:1010A00093F5828883E4737402936860EFA3A3A32B
:1010B00080DFD083D082F8E4937012740193700DB6
:1010C000A3A393F8740193F5828883E47374029365
:1010D000B5F0067403936860E9A3A3A3A380D8F9CD
:1010E00022C002C004C00612FFF0D006D004D00215
:1010F0002201670002530000020A000200AD07ED62
:101100002402F8E6F9A805E6FE08E6FBAA0675B192
:101110001053B33F53B2BF7803CEC313CE13D8F9E5
:10112000F5BCEBAE027805C333CE33CED8F9F5BDAE
:10113000E4F5BFFFEFC399500BED24032FF8E6F55C
:10114000A30F80F0E92440F5B3E5B230E6FB227549
:1011500044057545C0754608E4FF745F2FF8E6FE48
:1011600074472FF8A6060FBF08F07F44808FE4F580
:101170002FE55754E0FFC4135407F52CD28EE4F545
:1011800053F554E52C64016008E52C6402600241CB
:10119000D4E4F52E7458252EF8E6FF7460252EF859
:1011A000A607052EE52EB403EBE559FE7C00E425E9
:1011B00058F550EC3EF54F855A52E550854FF011E9
:1011C000B211D9100011F71001120B1018124D1F97
:1011D00050127D1F51000012C8E52CB40102418657
:1011E000E552600241C8755F4375634275644F758F
:1011F000654F7566544196E52CB401024186E5526F
:10120000600241C8755F4FF5634196E52CB4010259
:101210008074E5527008755F4F7563028078E552FF
:10122000B40111755F43756341756453756545E499
:10123000F5668062E5526402600241C8755F4375DD
:10124000634175645475654D75664C8049E552700F
:101250000FE52CB40102802E755F4F756301803657
:10126000E55264017062E52CB402028039755500C4
:10127000755602E4F567F107752FFF804BE5527054
:101280001AE52CB4010A7F067E017D007C0261B262
:10129000755F4F756301314F7FFF22E55264017026
:1012A00027E52CB4020A7F067E017D007C0161B235
:1012B000755F60314FE55BB4010BE4F5A775A61EC1
:1012C00075A6E180FE7FFF22E52F70087F067E0273
:1012D000FDFC61B2E52C64017024755102F52D7599
:1012E0005F60752E04B15EB408FBE52D6010E4F577
:1012F0002EE52EC3952D5006745BB16A80F3E52C64
:101300007071E551640260067D00B14161B2E5573C
:10131000541065677053E557540EC313FFC3740729
:101320009FF52DE5672420F55F752E01B15EB408A9
:10133000FBE55064507004E54F641F7010E552B433
:10134000010B7D58AF2D71B7EF70128020E4F52EA0
:10135000E52EC3952D50067458B16A80F3E55730D9
:10136000E011E4F551C28E800A7E03D19BF551C293
:101370008EFF22E52C64016004E52C7020314FE5DE
:101380002D2556F556E43555F555E52C700CE567D9
:1013900070057567108003E4F5677FFF22E52CB4C4
:1013A000040AE4F551C28EF5677FFF22E4F551FD92
:1013B000B141B1147F00228F308D31E53070037F51
:1013C0000122E4F532E532C395304002A10AE5314D
:1013D0002532F874D026F6E6FFD394104017EF9428
:1013E00031E53150092532F874F926F680072532A7
:1013F000F874D926F6E508118C1424001439011468
:101400004502145803146404147705148306149ECB
:101410000714A30814BF0914CB0A14EA0B14F60C22
:1014200000001506B10D640A6002A106750A007578
:101430000B02F50E750801A106B10DC454F0F509B3
:10144000750802A106B10D4209E509B14AE50B7024
:1014500002050A750803A106B10DC454F0F53575EF
:101460000804A106B10D4235E535B154E50B700213
:10147000050A750805A106B10DC454F0F5367508C6
:1014800006A106B10D4236E536B154E50B700205F2
:101490000AE535F50CE536F50D7508078068750821
:1014A000088063B10DB401028036E509D394105071
:1014B00004E50970307F087E007D00C1568026B1AA
:1014C0000DC454F0F53375080A803BB10D4233E585
:1014D00033B14AE50B7002050A050EE50EB50905A4
:1014E00075080B8021750809801CB10DC454F0F5F6
:1014F0003475080C8010B10D4234E4F508AF34B1F6
:101500007FEF7002FF22053261C57F0122E53125A0
:1015100032F8E6228F438E428D418C40E4F56775A8
:101520005F80E550F560E54FF561855262E4FF7438
:10153000402FF8E6FE74632FF8A6060FBF04F021D3
:101540004FC28E7F057E047C0122850B82850A8333
:10155000F0050B22850B82850A83F0050B22745F50
:10156000252EF8E4F6052EE52E22252EF8E6FFE5D9
:1015700056252EF582E43555F583EFF0052E22E44D
:10158000FE753700753802E50970037F0122E4FD1E
:10159000FCE5092403FBE433FAC3ED9BEC9A5019F4
:1015A0000538E538AA377002053714F5828A83E0DA
:1015B0002EFE0DBD00010C80D8C3E49E6F60087F35
:1015C000087E007D008035850C39E50D5480F53AA4
:1015D000AF097E00E50D2509CFEE350CCF24FFF5D0
:1015E0003FEF34FFF53EF53BE53F5480F53CE539F0
:1015F000131313541F640270057F08FD8058E53AE9
:10160000B53C08E539B53B03D38001C392003000F7
:101610000585093D8007C3E53C950DF53D74022421
:1016200003FDE43400FCAB3DAF0DAE0CD173D15DD6
:1016300020002074022403FFE43400FE7C00EF2528
:101640003DFDEC3EFCE53F547F04FBAF3CAE3BD19F
:1016500073D15D7F01227C20B1147F002243890178
:10166000758C63758AC4D28C308DFDC28CC28D534B
:1016700089F0228B4085A24153A2FE8E838F820582
:10168000A28C838D82740911DFE54053A2FE43A230
:101690002011E153A2DF8541A2FF227F057D007C5E
:1016A00000B114E422C3E5549466E5539400400E5F
:1016B000E551600AC28EC28F7E04D19BF551308FF6
:1016C00014C28F0554E554700205534553700674D7
:1016D000FFF553F55422E4F5B1E5B230E5277F215B
:1016E000F168E523B4081EE522B44019E521B406EB
:1016F00014E4FF74242FF8E6FE74572FF8A6060FA3
:10170000BF08F0316E809EE4F50822758F01F11656
:10171000F14FD1D680FC75B41275B50A75B61CE4CC
:10172000F5B175BCC8F5BDF5BF75C4FF75C5FF75CE
:10173000C705F5B275B38875AB02E5AA30E2FB7553
:101740002107752240752301E4F5247F2101FDE482
:10175000FF74572FF8E4F6745F2FF8E4F60FBF0814
:10176000F0E4F55143891022AD07AFBCEF75F008E6
:10177000A4FFE5BDC4135407FBEF4BA805A6F00872
:10178000F6E5B3540FFFED2402F8A607E4FFED24BD
:1017900002F8E6FEEFC39E500AED24032FF8A6A33D
:0C17A0000F80EB53B2DF75B3887FFF228F
:00000001FF
